:0200000480007A
:100000006F000005732F2034930F80006308FF03F7
:10001000930F90006304FF03930FB0006300FF038E
:10002000130F000063040F0067000F00732F2034CC
:1000300063540F006F00400093E19153171F0000BD
:1000400023223FFC171F000023200FFC6FF01FFF2F
:100050009300000013010000930100001302000050
:100060009302000013030000930300001304000038
:100070009304000013050000930500001306000020
:100080009306000013070000930700001308000008
:10009000930800001309000093090000130A0000F0
:1000A000930A0000130B0000930B0000130C0000D8
:1000B000930C0000130D0000930D0000130E0000C0
:1000C000930E0000130F0000930F0000732540F102
:1000D0006310050097020000938202017390523072
:1000E000735044749702000093820201739052305F
:1000F00073500018970200009382420273905230AE
:100100009B021000939252039382F2FF7390023B82
:100110009302F0017390023A73504030970200004E
:1001200093824201739052307350203073503030BC
:100130009301000097020000938202ED7390523009
:10014000130510001315F501635C05000F00F00F97
:10015000930110009308D005130500007300000000
:1001600093020000638A020073905210B7B200003D
:100170009B829210739022307350003097020000DF
:100180009382420173901234732540F17300203042
:1001900093012000B70001FF9B8000F013E7F0F00F
:1001A0009303F0F0631C771C93013000B710F00F3D
:1001B0009B8000FF13E7000FB713F00F9B8303FF33
:1001C000631E771A93014000B700FF009B80F00F79
:1001D00013E7F070B703FF009B83F37F6310771A78
:1001E00093015000B7F00FF09B80F00013E7000F71
:1001F000B7F30FF09B83F30F63127718930160003E
:10020000B70001009B8010F093900001938000F0F4
:1002100093E0000FB70301009B8313F09393030156
:10022000938303FF639C701493017000130200001A
:10023000B710F00F9B8000FF13E7000F13030700B8
:100240001302120093022000E31452FEB713F00FC2
:100250009B8303FF63147312930180001302000059
:10026000B700FF009B80F00F13E7F0701300000051
:10027000130307001302120093022000E31252FE40
:10028000B703FF009B83F37F631A730E9301900003
:1002900013020000B7F00FF09B80F00013E7000F8F
:1002A00013000000130000001303070013021200E4
:1002B00093022000E31052FEB7F30FF09B83F30F7D
:1002C000631E730A9301A00013020000B710F00F21
:1002D0009B8000FF13E7000F13021200930220001F
:1002E000E31652FEB713F00F9B8303FF63187708E2
:1002F0009301B00013020000B700FF009B80F00FD5
:100300001300000013E7F0F0130212009302200024
:10031000E31452FE9303F0FF631277069301C000CB
:1003200013020000B7F00FF09B80F00013000000F4
:100330001300000013E7000F1302120093022000C5
:10034000E31252FEB7F30FF09B83F30F63187702AB
:100350009301D0009360000F9303000F639070022D
:100360009301E000B700FF009B80F00F13E0F070F6
:100370009303000063147000631030020F00F00F4D
:10038000638001009391110093E111009308D0055F
:1003900013850100730000000F00F00F930110009F
:1003A0009308D0051305000073000000731000C00F
:0C03B00000000000000000000000000041
:1010000000000000000000000000000000000000E0
:1010100000000000000000000000000000000000D0
:1010200000000000000000000000000000000000C0
:1010300000000000000000000000000000000000B0
:081040000000000000000000A8
:040000058000000077
:00000001FF
